:100000000C9491020C94AE020C94AE020C94AE02CD
:100010000C94AE020C94AE020C94AE020C94AE02A0
:100020000C94AE020C94AE020C947C1D0C944E1EEB
:100030000C9462180C94AE020C94AE020C94AE02B6
:100040000C94AE020C94AE020C94AE020C94AE0270
:100050000C94AE020C94EA180C94AE020C94AE020E
:100060000C94AE020C94AE020C94AE020C94AE0250
:100070000C94AE020C94AE020C94AE020C94AE0240
:100080000C94AE020C94AE020C94AE020C94AE0230
:100090000C94AE020C94AE020C94AE020C94AE0220
:1000A0000C94AE020C94AE020C94AE02D604D604AC
:1000B000020502056A058805A006A00693052C0620
:1000C0003D063D06BB1EE21EDA1FE21EDA1F2E1F92
:1000D000511FDA1FA81FB71F290000003A003B007C
:1000E0003C003D0000003E003F0040004100350064
:1000F0001E001F00200021002200230024002500F4
:10010000260027002B0014001A0008001500170015
:100110001C0018000C001200130000000400160060
:10012000070009000A000B000D000E000F0033004D
:10013000E10000001D001B00060019000500110071
:10014000100036003700E000E3000000E20000008D
:1001500000002C0000000000000001510000000021
:1001600000000000480047004600450044004300EE
:10017000420056005500540053004B004A0049000D
:1001800000002A002E002D000000610060005F00CA
:100190004E004D004C003100000030002F00570091
:1001A0005E005D005C000000000000000000280010
:1001B0000000340000005B005A00590000005200AB
:1001C00000000000E5000000380058006300000057
:1001D00062004F0051005000E000000065780251BD
:1001E000005C0000010001000100010000000100AE
:1001F00001000100010001000100010001000100F7
:1002000001000100010001000100010001000100E6
:1002100001000100010001000100010001000100D6
:1002200001003900AC00AD00AE00AB0001000100E0
:100230000100010001000100010000000100AA000E
:10024000A900A80001000100010001000100010057
:10025000010000000100000000000100000000009B
:10026000000001000000000000000000010001008B
:100270000100010001000100010001000100010076
:10028000010001004A01010000004C0001000100D2
:100290000000010001000100010001000100010057
:1002A0000000010001000100010001000100000048
:1002B000000000000000010000000100000001003B
:1002C000010001000000010000000000010000002A
:1002D0000100010001000000010001000100010017
:1002E0000100000001000100005C000001000100AD
:1002F0000100010000000100AA00A900A8000100FF
:1003000001000100010001000100010001000100E5
:1003100001000100010001000100010001000100D5
:1003200001000100010001000100010001000100C5
:100330000100010001005000510052004F00010077
:1003400001000000010001000100010001000100A6
:100350000100010001000100010000000100000097
:10036000000001000000000000000100000000008B
:1003700000000000010001000100AB00AE00AD0074
:10038000AC000100010001000100010001000100BA
:100390000000010001000100000001000100010057
:1003A0000100010001000100000001000100010046
:1003B0000100010001000000000000000000010039
:1003C0000000010000000100010001000000010028
:1003D0000000000001000000010001000100000019
:1003E0000100010001000100010000000100010006
:1003F0001C035200650064007200610067006F001A
:100400006E002000560061007200610000000603CB
:100410005000480000000403090409023B000201E7
:1004200000A0FA09040000010301010009211101E3
:1004300000012240000705810308000109040100B2
:100440000103000000092111010001227B000705C2
:100450008203200001120100020000000848500140
:100460000001000102000105010902A10185020944
:1004700001A1000509190129081500250195087534
:100480000181020501093009311581257F95027529
:1004900008810609381581257F95017508810605B3
:1004A0000C0A38021581257F950175088106C0C0A8
:1004B00005010980A101850319012AB7001501264C
:1004C000B700950175108100C0050C0901A10185D7
:1004D0000419012AA002150126A0029501751081B8
:1004E00000C005010906A101050719E029E715006B
:1004F000250195087501810295017508810105079F
:10050000190029FF150026FF0095067508810005D2
:100510000819012905950575019102950175039149
:1005200001C011241FBECFEFDAE0DEBFCDBF11E066
:10053000A0E0B1E0EAE1F1E402C005900D92A23939
:10054000B107D9F722E0A2E9B1E001C01D92AC3CAD
:10055000B207E1F70E94AB120C948B200C940000C0
:1005600081E0089581E008950C94B20208950C94FE
:10057000B6021F93CF93DF9300D000D01F92CDB768
:10058000DEB749835A836B833091950189819A81C3
:10059000311114C0662359F0222349F00E94DD086E
:1005A000182F682F89819A810E94860803C00E94B3
:1005B000B108182F69817A81812F04C00E94DD085B
:1005C00069817A810F900F900F900F900F90DF91BB
:1005D000CF911F910C941310FC01262F4081518163
:1005E0006281738184810C94B90281E00895CF9374
:1005F000DF93EC0160E00E94EC02BE01DF91CF913D
:100600000C94B7020C945C110C94581108950E943C
:1006100030070E9406032FEF84E39CE021508040C6
:100620009040E1F700C000000C9410190F931F9345
:10063000CF93DF938C0161E00E94EC02EC01B801E2
:100640000E94B4028823F1F1B801CE010E942D1757
:100650008823C1F1B801CE010E944115882391F190
:10066000B801CE010E948916882361F1F8018281C8
:10067000882309F1CB358DE5D807C1F050F4C115B9
:10068000FCE5DF0781F0CF3DDC45A9F40E94140EA4
:1006900019C0CC35EDE5DE0761F0CD35DD4559F407
:1006A0000E94570D08C00E9407030CC00E94600DF5
:1006B00002C00E94630DC801DF91CF911F910F917D
:1006C0000C94B00280E0DF91CF911F910F910895BB
:1006D0000E9444180C9481030E9484030C944A18CD
:1006E00008950C94700381E008950C9473030895A9
:1006F000CF93C82F0E9471038C2F0E947503CF9156
:10070000089580E00C9478030E9489170C94780374
:100710000E94891790919401891721F08093940188
:100720000C9478030895CF93DF93CDB7DEB72B9762
:100730000FB6F894DEBF0FBECDBF4F8358876987D1
:100740007A878B8761110E94A30C9E012F5F3F4F18
:1007500086E0F90111928A95E9F785E0FE01379666
:10076000D90101900D928A95E1F789819A814C8196
:100770005D81452B31F09F3F31F491E08F3F19F4BB
:1007800003C091E001C090E090FF09C049815A8107
:100790006B817C818D819E810E94C40B05C0C90143
:1007A0000E94F5028111F2CF2B960FB6F894DEBFAE
:1007B0000FBECDBFDF91CF910895FC018081918163
:1007C0000E941F090895CF93882309F450C0C82FB1
:1007D0008CEF8C0F813AD0F46C2F809102019091B4
:1007E00003010E94E617882349F06C2F80910201D3
:1007F000909103010E941E180E94C50C6C2F8091DD
:100800000201909103010E941C180CC080E28C0F21
:10081000883058F4C77081E001C0880FCA95EAF7A4
:100820000E94860CCF910C94C50CEBE5EC0FE330E5
:1008300040F4F0E0E95BFE4F808190E0CF910C94B2
:10084000AE17E8E5EC0FE73150F4F0E0EE0FFF1FD4
:10085000E75EFE4F80819181CF910C94C417CD3E0D
:1008600030F08C2F0E943013CF910C940214CF9152
:100870000895882389F19CEF980F913A40F4682FEE
:1008800080910201909103010E941E180DC090E218
:10089000980F983058F4877091E001C0990F8A95AD
:1008A000EAF7892F0E948C0C0C94C50C9BE5980FDD
:1008B000933020F480E090E00C94AE1798E5980F08
:1008C000973120F480E090E00C94C4178D3E20F026
:1008D0000E948B130C94021408951F93CF93DF93FF
:1008E000182FEB010E94E303209741F08FE99FE06E
:1008F0000197F1F700C000002197F6CF812FDF911B
:10090000CF911F910C943904893319F060E070E0A5
:1009100002C060E570E00C946D04882321F00E9411
:10092000860C0C94C50C0895882321F00E948C0C31
:100930000C94C50C0895CF92DF92EF92FF920F9323
:100940001F93CF93DF937C01D62FC72FFC01128119
:10095000058102950F700E947C0C8823B9F0112349
:10096000A9F08C2F807F803421F080E28D0F8830B9
:1009700068F080918A0282FD09C082E00E94250D04
:100980000E947C0C91E0D82ED92601C0D12CCC2E0F
:10099000C2948FE0C8228C2D90E08C30910508F035
:1009A000CFC1FC01EA5AFF4F0C9422208C2F807F8C
:1009B000CF70882311F0C295C07F112399F0CC230A
:1009C00009F4AAC180E28D0F883010F0D11104C063
:1009D0008C2F0E94860C03C08C2F0E94960C0E94C4
:1009E000C50C9AC18D2F0E943904CC2309F4A8C1EB
:1009F00080E28D0F883038F1DD2329F18C2F0E94A1
:100A00009C0C24C08C2F807FCF70803211F0C29557
:100A1000C07FDD2319F0D130A1F13DC080918A0261
:100A200082FF17C0112349F0CC2329F08C2F0E949C
:100A3000860C0E94C50C80E070C180E00E943904E1
:100A4000CC2309F47DC18C2F0E948C0C0E94C50C14
:100A500077C1112371F0002341F0013031F40E947D
:100A6000A60C8C2B0E94AE0C6BC10E94A60C8C2B8A
:100A70001DC0002319F0013009F462C10E94BB0CB3
:100A800025C0112321F0063008F05AC10EC00530F0
:100A900008F056C11BC0112361F0002331F0F701AB
:100AA000858180FF39C18F7085838C2F0E948D04D2
:100AB00047C1002359F0D93309F03FC1FFEF07EEDA
:100AC00013E0F15000401040E1F735C18C2F0E9437
:100AD000940436C18C2F86958695837019F08130E9
:100AE00061F02EC1112321F08D2F9C2F937002C035
:100AF00080E090E00E94AE172BC1112321F08D2FD2
:100B00009C2F937002C080E090E00E94C41720C127
:100B10008D2F112319F00E94301302C00E948B13F5
:100B20000E94021415C18C2F837009F047C0111167
:100B30000BC12D2F229526952770220F220F6D2F86
:100B40006F70862F90E0A0E0B0E0022E04C0880F06
:100B5000991FAA1FBB1F0A94D2F7D4FF10C04FE001
:100B600050E060E070E004C0440F551F661F771F1F
:100B70002A95D2F7409550956095709503C040E056
:100B800050E0BA01C695C695C3708A019B01082B37
:100B9000192B2A2B3B2BC901B801C23049F058F45C
:100BA000C13019F00E949C07CFC00E948A07CCC0B8
:100BB0000E94AE07C9C00E948807C6C0112319F061
:100BC0008C2F817001C08695882309F4BDC02D2F1C
:100BD000229526952770220F220F6D2F6F70862F7A
:100BE00090E0A0E0B0E0022E04C0880F991FAA1F79
:100BF000BB1F0A94D2F7D4FF10C04FE050E060E072
:100C000070E004C0440F551F661F771F2A95D2F766
:100C1000409550956095709503C040E050E0BA0152
:100C2000C695C695C3708A019B01082B192B2A2BE8
:100C30003B2BC901B801C23049F058F4C13019F05A
:100C40000E94610881C00E944F087EC00E94730804
:100C50007BC00E94C20778C0CF70112339F08C2F5F
:100C60000E94E8078D2F0E948D046EC08D2F0E9478
:100C700094048C2F0E94090867C0D23F21F128F408
:100C8000D03F41F0D13FC1F043C0D33F19F1D43F31
:100C900079F03EC0112341F0053008F051C08C2F8F
:100CA0008F710E942E084CC0063008F049C0F7CF63
:100CB00080918A0282FF18C0112339F08C2F8F7126
:100CC0000E94E8073DC01123C9F38C2F8F710E9449
:100CD000090836C0112329F08C2F8F710E94D30789
:100CE0002FC00E94CE072CC0112349F0CF718C2F4A
:100CF0000E94E80763E08C2F0E940A0D21C081E06A
:100D00000E94250D0230E0F082E00E94250D18C0FF
:100D1000112331F0002391F28D2F0E94E30310C0C4
:100D2000002399F2D93349F41FEF27EE33E0115035
:100D300020403040E1F700C000008D2F0E943904B0
:100D400088EF8C0D843020F40E9489170E9478036C
:100D5000DD20C9F00E94780C80FD15C0F7011282D9
:100D60000E94720C0E94E807C7010E94E4060E94DC
:100D7000720CDF91CF911F910F91FF90EF90DF9058
:100D8000CF900C940908DF91CF911F910F91FF90A4
:100D9000EF90DF90CF9008950F931F93CF93DF9341
:100DA000EC01688179818A810E942A098C010E9464
:100DB00085080E947607B801CE010E949B04DF914E
:100DC000CF911F910F910895CF93DF93EC019881FC
:100DD00089812B813C81232B31F08F3F31F481E0DD
:100DE0009F3F19F403C081E001C080E080FD1DC079
:100DF000CE010E941603811110C00E947C0C882332
:100E0000A1F08A81882389F080918A0282FD0DC039
:100E100082E0DF91CF910C94250DCE010E94CC068B
:100E2000CE01DF91CF910C94F702DF91CF9108951D
:100E300080E090E00E94AE1780E090E00E94C4172E
:100E40000E94A30C0E94C50C0E9433150C9402143E
:100E500080910201909103010E9420180C941807C0
:100E60000E94930C0C94280792959F70963079F00D
:100E700010F4925001C09A50923068F4803F69F0AB
:100E800018F4883E40F409C0843F29F406C0883E27
:100E900020F0813F11F080E0089581E00895FC0189
:100EA000808191810E941F090E9434070895CF9389
:100EB000DF9300D000D01F92CDB7DEB70F900F9018
:100EC0000F900F900F90DF91CF910895CF93DF9304
:100ED00000D000D000D0CDB7DEB726960FB6F8947C
:100EE000DEBF0FBECDBFDF91CF9108950895089565
:100EF0000C9477070C9478070E947A076093EF01AF
:100F00007093F0018093F1019093F2010C94180713
:100F10000C947C070F931F930091EF011091F00147
:100F20002091F1013091F201602B712B822B932BD8
:100F30001F910F910C947C070F931F930091EF0169
:100F40001091F0012091F1013091F20160237123A1
:100F5000822393231F910F910C947C070F931F936F
:100F60000091EF011091F0012091F1013091F20117
:100F700060277127822793271F910F910C947C077C
:100F80000C9477070E94C0076093EB017093EC010B
:100F90008093ED019093EE010C94180760E070E0EF
:100FA000CB010C94C2070F931F9341E050E060E027
:100FB00070E08A019B0104C0000F111F221F331F24
:100FC0008A95D2F7C901B8011F910F910C94C207FD
:100FD0000F931F9341E050E060E070E004C0440FC5
:100FE000551F661F771F8A95D2F78091EB0190916C
:100FF000EC01A091ED01B091EE018A019B01082B5B
:10100000192B2A2B3B2BC901B8011F910F910C946E
:10101000C2070F931F9341E050E060E070E004C00E
:10102000440F551F661F771F8A95D2F7409550953C
:10103000609570958091EB019091EC01A091ED018C
:10104000B091EE018A019B01082319232A233B2337
:10105000C901B8011F910F910C94C2070F931F9300
:1010600041E050E060E070E004C0440F551F661F8F
:10107000771F8A95D2F78091EB019091EC01A091B6
:10108000ED01B091EE018A019B01082719272A275B
:101090003B27C901B8011F910F910C94C2070F9310
:1010A0001F930091EB011091EC012091ED01309123
:1010B000EE01602B712B822B932B1F910F910C94BF
:1010C000C2070F931F930091EB011091EC01209147
:1010D000ED013091EE0160237123822393231F9150
:1010E0000F910C94C2070F931F930091EB01109185
:1010F000EC012091ED013091EE01602771278227EC
:1011000093271F910F910C94C20708952BE0929F93
:10111000800D1124E82FE695E695E695877051E05D
:1011200001C0550F8A95EAF785E0E89FF001112488
:10113000EA56FE4F20E030E070E04081CB01022E05
:1011400002C0969587950A94E2F78170819584276D
:101150008523842781932F5F3F4F2530310569F721
:1011600008952BE0929F800D1124682F6695669557
:101170006695982F977085E0689FB001112440E034
:1011800050E080E0FB01E40FF51FEA56FE4F20819E
:1011900030E0092E02C0369527950A94E2F72170B7
:1011A0003327042E01C0220F0A94EAF7822B4F5FE7
:1011B0005F4F4530510531F70895BF92CF92DF92CE
:1011C000EF92FF920F931F93CF93DF938C01C09008
:1011D000EB01D090EC01E090ED01F090EE018091F8
:1011E000EF019091F001A091F101B091F201C82AB4
:1011F000D92AEA2AFB2ACFE1D0E0D701C6010C2E7A
:1012000004C0B695A795979587950A94D2F780FD67
:1012100004C0219790F7B12C07C0BC2EB8018C2FC9
:101220000E9426100197A9F38B2DDF91CF911F917A
:101230000F91FF90EF90DF90CF90BF900895CF93E4
:10124000DF93EC010E94DD08BE010E942610DF91B1
:10125000CF9108951F93CF93DF93EB019091950168
:10126000992321F0CB010E941F0913C0882349F064
:10127000CB010E94DD08182F682FCE010E9486083E
:1012800004C0CB010E94B108182FBE01812F0E941B
:101290002610DF91CF911F9108951F93CF93DF9375
:1012A000C091F30116E08091F401C81799F0D0E0E5
:1012B0001C9FF0011D9FF00D1124EB50FE4F40814B
:1012C000518162817381848195810E946607219694
:1012D000C770E9CFDF91CF911F910895409125020A
:1012E0005091260260912702709128028091290274
:1012F00090912A020C946607EF92FF920F931F932E
:10130000CF93DF9380912A0282958F7009F065C098
:1013100080912702882309F460C08091F301F09046
:10132000F40110912502009126026091280270912B
:10133000290291E01F3F09F090E0C0910001D09197
:101340000101292F96E0E92E8F1509F446C0611599
:10135000710521F00F3F21F030E003C031E001C002
:10136000322F90E030FD36C0E89EF001E99EF00D8E
:101370001124DF01AB50BE4F11963C9111973013F1
:1013800029C03C91311326C012963C91129731111D
:1013900021C013964D915C911497461B570B4C1727
:1013A0005D07C0F480912A028F70806180932A02C9
:1013B000E650FE4F80818F708061808385E292E0ED
:1013C0000E94E406DF91CF911F910F91FF90EF9063
:1013D0000C944D0901968770B7CFDF91CF911F9183
:1013E0000F91FF90EF9008959F92AF92BF92CF928E
:1013F000DF92EF92FF920F931F93CF93DF93CDB7BE
:10140000DEB761970FB6F894DEBF0FBECDBF8C017B
:1014100085E0F801DE011D9601900D928A95E1F7B5
:10142000D8011296EC9090912502E091260220912D
:101430002802309129022115310531F0EF3F31F4B6
:1014400081E09F3F19F403C081E001C080E0B82F24
:10145000B1709B2E80FD47C1D8014C9111965C91D3
:1014600011971396AD90BC90149785E2C82E82E038
:10147000D82EF0902702B501621B730B209100015A
:1014800030910101FF2009F4D9C080912A0262172E
:10149000730708F095C0282F207F09F052C05E1313
:1014A00013C0491311C0FE2CE1100EC08F70806173
:1014B00080932A020E946E09C6010E94E406809170
:1014C0002A02F80185834DC1AB2831F05F3F31F42A
:1014D00081E04F3F19F403C081E001C080E080FD4E
:1014E00003C081E08E2502C080E090E0F82FF1700B
:1014F000FF2E80FF1CC08091F3012091F40136E0A3
:10150000821709F40BC190E0389FF001399FF00D6C
:101510001124EB50FE4F6181561306C060814613C3
:1015200003C06281E61203C001968770E9CFFE2CEA
:10153000EE2009F416C180912A02816080932A026C
:1015400054C05E1306C0491304C0E11002C0F80184
:1015500099C0C8010E944F07882361F1EE2051F124
:1015600020912A02822F82958F7090E0029774F06A
:10157000809125029091260298878F831986BB86D9
:10158000AA862C87CE0107960E94E40686E0F80121
:10159000A5E2B2E001900D928A95E1F70E947C09E4
:1015A0000E946E090AC05E1711F1C8010E944F0720
:1015B00081112CC0C8010E94E406FF24F394D1C01D
:1015C000282F207F81F77A2DB98AA88A6E2D8989E4
:1015D0000E94570785E292E00E94E40686E0D60169
:1015E0001D928A95E9F70E946E09F12CBAC0491341
:1015F000DCCFE110DACFF8018583C8010E94E40650
:1016000086E0D6011D928A95E9F7ABC0EE2091F2F3
:1016100020912A02822F82958F7090E002970CF41D
:10162000B5CF80912502909126029A8389831B82EF
:10163000BD82AC822E83CE010196A6CF62177307BE
:1016400008F044C0FE2CEE2009F4B4CF5E1330C085
:1016500049132EC020912A0220FD21C0822F82959D
:101660008F70482F50E041155105C9F0F8012583CE
:101670004F30510541F08F5F982F9295907F822FC8
:101680008F70892B8583C8010E94E40686E0F801EB
:10169000A5E2B2E001900D928A95E1F73CC086E0A8
:1016A000F801A5E2B2E001900D928A95E1F759C0E8
:1016B000C8010E944F07811169CF80912A02816081
:1016C00080932A02C8010E94E4064BC07A2DB98A91
:1016D000A88A6E2D89890E94570786E0D6011D923F
:1016E0008A95E9F718C0EE2009F464CFC8010E947A
:1016F0004F07F82E882309F45DCF86E0F801A5E2B4
:10170000B2E001900D928A95E1F785E292E00E94A5
:10171000DD030E947C090E946E0923C04D875E870D
:101720008D859E850E941F09292F22952F702230BA
:1017300028F49F7039F0811105C00BC0243028F4C3
:101740009F7049F4805E883020F0C8010E94E40652
:101750009F2CF92C06C0D80115969C91907F91F78B
:10176000F8CF8F2D61960FB6F894DEBF0FBECDBFB8
:10177000DF91CF911F910F91FF90EF90DF90CF906D
:10178000BF90AF909F9008951F93CF93DF93CDB7F5
:10179000DEB72C970FB6F894DEBF0FBECDBF4F83D8
:1017A000588769877A878B879C87CE0107960E9426
:1017B000F4098823D1F09F8188852A853B85232BD6
:1017C00031F08F3F31F481E09F3F19F403C081E095
:1017D00001C080E080FD47C04F81588569857A85CA
:1017E0008B859C850E9466073EC086E0FE01379689
:1017F000DE01119601900D928A95E1F7FF81E8854F
:101800006A857B856115710531F0EF3F31F481E028
:10181000FF3F19F403C081E001C080E080FD23C0D8
:101820002091F40130E0C901019687709927409119
:10183000F30150E084179507F1F1F983EA837D8382
:101840006C8396E0929FD001939FB00D1124AB5012
:10185000BE4FFE01319601900D929A95E1F780936B
:10186000F4010E944D0916E08091F3019091F4017A
:10187000891771F1189FC00111248B509E4F0E944F
:10188000F409882329F1E091F3011E9FF00111244E
:10189000EB50FE4F4081518162817381848195813B
:1018A0000E9466078091F30190E001968770992766
:1018B0008093F301D9CF0E9430071092F401109267
:1018C000F301E5E2F2E086E0DF011D928A95E9F797
:1018D0002C960FB6F894DEBF0FBECDBFDF91CF912F
:1018E0001F9108958091330285958595859508957A
:1018F000809133028770089590913302977081E050
:1019000009F480E0089580913E02089590913E028E
:10191000892B80933E020895809590913E02892301
:1019200080933E02089510923E02089590913D02E8
:10193000892B80933D020895809590913D028923E3
:1019400080933D02089510923D02089580913402E3
:10195000089508950C94A90C0C94AA0C90918A02F5
:1019600092FD08C090913402981721F080933402C0
:101970000C94AC0C089580913402882329F01092C5
:10198000340280E00C94AC0C0895CF93DF93E09187
:101990000201F091030180913E028083E0910201F7
:1019A000F0910301908180913D02892B8083809189
:1019B0003402882381F0E0910201F09103019081CB
:1019C000892B808380910201909103010E94DA1794
:1019D00081110E94BB0CC0910201D091030148E02B
:1019E00050E06BE272E0CE010E943C20892B69F04E
:1019F00088E0FE01ABE2B2E001900D928A95E1F73A
:101A0000CE01DF91CF910C949517DF91CF9108957E
:101A10000C94A90C90918A0292FD10C098E0899FC5
:101A200090011124262B209333020E94E807809115
:101A300033028595859585950C94080D0C94E807DF
:101A40001092330280E00C94080D209133028095AF
:101A5000822380933302982F977099F430E0482FB7
:101A6000082E000C550B2417350759F090918A0267
:101A700092FD07C08595859585950E9409080C946F
:101A8000200D089590918A0292FB222720F92817B1
:101A900069F080FB92F990938A028091890290917B
:101AA0008A020E94900D82E00C94250D0895809189
:101AB0008A0282FB882780F991E089270C94420DE5
:101AC00081E00C94420D80E00C94420D6FEF7FEFAB
:101AD00080E090E00C94752080E090E00E9451201E
:101AE00021E0893E9E4F09F020E0822F089582E098
:101AF00090E00C94492083E090E00C944920CF932F
:101B000084E090E00E944920C82F82E290E00E9489
:101B100049202C2F30E0A901582BCA01CF910895FC
:101B2000CF93C92F682F84E090E00E9457206C2F3C
:101B300082E290E0CF910C945720AB01BC018FE082
:101B400090E00C946920AB01BC0183E190E00C941F
:101B5000692060E070E0CB010C94A30D60E070E0C0
:101B6000CB010E949D0D0C94A90D69EE7EEF80E0E3
:101B700090E00E94752060E082E090E00E94572093
:101B800060E083E090E00E9457201092EF011092F5
:101B9000F0011092F1011092F20160E084E090E017
:101BA0000E94572060E082E290E00E94572060E0AF
:101BB00085E090E00E94572060E086E090E00E947F
:101BC00057206FEF87E090E00E94572040E050E000
:101BD000BA0188E090E00E94692060E08DE090E02A
:101BE0000E94572040E050E0BA0188E190E00E9456
:101BF000692060E087E190E00E94572040E050E0DB
:101C0000BA018CE190E00E94692060E070E080E21F
:101C100090E00E94752040E050E0BA0188E190E039
:101C20000E9469200C94AE0D0C94B50D682F8EE0C7
:101C300090E00C9457200E94CF1860935B02709341
:101C40005C0280935D0290935E02609357027093F2
:101C500058028093590290935A02089585B780687C
:101C600085BF85B7806885BF089581E008950C948D
:101C7000350E08950C94390E0C94390E0C943C0ECC
:101C80000C94390E0C94400E0C94390E0E942E0EBA
:101C900082E091E10E947F170E94440E0C94420E54
:101CA0000E943A0E0C94390E0E941F110C94770377
:101CB0000E94BA180E9404120E94540E0C943E0E08
:101CC0005F926F927F928F929F92AF92BF92CF92CC
:101CD000DF92EF92FF920F931F93CF93DF93CDB7D5
:101CE000DEB72A970FB6F894DEBF0FBECDBF0E94B5
:101CF0001912C82E81110E941B0E3FE3832E32E081
:101D0000932E00E010E0502E802F0E9443115C01C2
:101D1000F401619071904F01682679266114710475
:101D2000B1F40F5F1F4F0C30110569F78FEF8983F6
:101D30008A831B820E94C3188160782F9D838C83C5
:101D400049815A816B818D810E9493033AC08091B1
:101D50005F0281FD0E944C11D12CEE24E394F12C02
:101D6000C3018E219F21892B29F10E94370E8823E0
:101D7000A9F0DE825F82AE20BF2081E0AB2809F4AB
:101D800080E088870E94C3188160782F9A878987AE
:101D90004E815F8168858A850E949303000F111F21
:101DA000F801E15CFD4F80819181E826F926F182FE
:101DB000E08207C0D394EE0CFF1CFBE0DF12D0CF13
:101DC000B0CF81E0C11001C080E02A960FB6F89430
:101DD000DEBF0FBECDBFDF91CF911F910F91FF905E
:101DE000EF90DF90CF90BF90AF909F908F907F90BB
:101DF0006F905F9008950E94600E0E9420140C94D2
:101E00008803CF93DF930E942B10EC01811521E50D
:101E1000920708F045C0811530E5930708F094C09B
:101E2000883E910528F5803E910508F0F8C0883A73
:101E3000910570F4853A910508F07CC081309105D8
:101E400009F475C008F4E8C0049708F0E8C0E4C0DD
:101E50008F3B910508F0E0C0C85AD0E0CC0FDD1FE1
:101E6000C65BDE4F0990D881C02DCE019464D8C0E6
:101E7000811540E2940758F4811551E0950708F068
:101E8000CEC08D3E910508F4C7C09065C9C0C1158C
:101E900080E4D80708F4C0C0DF70CE01906AC0C0EB
:101EA000811525E59207A8F4811534E5930708F01C
:101EB00095C0811543E5940708F07BC0811552E574
:101EC000950708F061C0D82FCC27CE01816F906AAA
:101ED000A7C0C11589E5D807A0F4C11528E5D20728
:101EE00008F082C0C11536E5D30708F095C08C2FE5
:101EF0000E94BF108F7190E0D82FCC27CE01906246
:101F00008FC0C1154AE5D40708F474C0CE019056BD
:101F10008115904208F080C08D2F8F710E94BF10F4
:101F2000DD27D0628F71AE01582BCA0179C081E0E4
:101F300090E076C0C55AD0E0C858DE4F8881C82FDF
:101F4000D0E0CE0190646CC074E0969587957A9548
:101F5000E1F7282F23703C2F337081E090E002C01E
:101F6000880F991F3A95E2F79C68AC01522B9A01B1
:101F70009C2F9F709695969550E2959FE0011124B5
:101F8000C9018C2B9D2B4CC08370992721E030E038
:101F900002C0220F331F8A95E2F79C2F96959695E3
:101FA00080E2989FE0011124C22BD32BCE019C68C4
:101FB00037C08370992721E030E002C0220F331F21
:101FC0008A95E2F79C2F9695969540E2949FE001C2
:101FD0001124C22BD32BCE019A6822C0D82FCC2734
:101FE000CE01846F906A1CC0DC2FCC27CE01806F9D
:101FF000906A16C08C2F8F700E94BF1094E0D69507
:10200000C7959A95E1F7CF70D0E0DC2FCC27D06947
:102010009E01282BC90104C080E090E001C0CE01E0
:10202000DF91CF91089524E8829FC0011124FC0123
:102030002BE0729FE00DF11D1124E60FF11DEE0F54
:10204000FF1FE852FF4F8591949108950E9413104D
:102050000E94010F08958238910569F1B0F481332F
:10206000910509F46DC048F48932910509F463C003
:102070008A32910509F469C008958533910509F400
:1020800055C089339105B9F00895833E910569F1F2
:1020900038F4803E9105B1F0823E910509F1089532
:1020A000863E9105A9F1873E9105B9F1843E9105DF
:1020B00009F064C023C02091890220FD4FC021FD9A
:1020C0004DC008958091890280FD44C080918A02AC
:1020D00080FF44C08091890284FD42C083EE4DC0E0
:1020E0008091890282FF38C0F5CF8091890282FDFC
:1020F00033C080918A0280FD31C0ECCF80918A028A
:1021000081FF32C08091890284FD2AC087EE35C0EC
:102110008091890283FF26C0F5CF8091890283FDDB
:1021200021C080918A0281FD1FC0ECCF809189027D
:1021300085FD1CC01DC08091890285FD19C016C097
:102140008091890286FD16C017C08091890286FDA4
:1021500013C010C089E311C082EE0FC080EE0DC025
:1021600080E00BC086EE09C084EE07C089E205C09E
:1021700085E303C08AE201C081E390E00895909175
:10218000890292FF0DC0282F2871283019F4877F0B
:10219000846006C0282F2471243011F48B7F88605E
:1021A00093FF0DC0282F2871283119F4877E846190
:1021B00006C0282F2471243111F48B7E8861209170
:1021C0008A0220FF0DC0382F3871383019F4877F0C
:1021D000816006C0382F3171313011F48E7F8860F4
:1021E00021FF0DC0282F2871283119F4877E8161C5
:1021F00006C0282F2171213111F48E7E886194FD53
:10220000877E089580E008950C94660D0E9419124F
:102210002FEF86E791E0215080409040E1F700C029
:1022200000000E94191280E00E94431180FF04C048
:102230000E9404110C94101908950C9406110E9428
:102240006C0D811102C00E94140E0E94770D8093C4
:102250005F020E947F0D90938A02809389020E9400
:102260001D110E947B0D682F70E080E090E00E94BD
:1022700088076091EB017091EC018091ED019091E4
:10228000EE010C94C007E82FF0E0EE0FFF1FED55B4
:10229000FD4F808191810895089580EA8A95F1F734
:1022A000089500C008950C944D1108950C94551193
:1022B0000C9456110C9455110C945A11F894E82F63
:1022C000E295EF70F0E031A1282F2F7081E090E0CF
:1022D00001C0880F2A95EAF7982F9095932391A330
:1022E00092A1892B82A3789408950F931F93CF9383
:1022F000DF93C6E8D1E089918F3F11F00E945E1113
:1023000081E0C239D807B9F7CBE7D1E006E811E0A0
:1023100089918F3F11F00E945E110C171D07C1F7C4
:10232000DF91CF911F910F910895BF92CF92DF92CD
:10233000EF92FF920F931F93CF93DF938C01C62FE1
:10234000D0E0CE018A579E4F6C01FC0190819F3FE7
:1023500009F450C0B62EF894E92FE295EF70F0E042
:1023600081A19F7021E030E001C0220F9A95EAF729
:10237000822B81A382A12095282322A378940E94F6
:102380005111EBE7F1E046E851E021E030E0E12CCB
:10239000F12C61916F3F89F0A62FA295AF70B0E04C
:1023A00090968C9190E06F7002C0959587956A9594
:1023B000E2F780FD02C0C90102C080E090E0E82A97
:1023C000F92A220F331F4E175F0719F7F601808194
:1023D0008F3F11F00E945E1161E0E114F10409F4F5
:1023E00060E08B2D0E945311CC0FDD1FC00FD11F59
:1023F000F982E882DF91CF911F910F91FF90EF90CA
:10240000DF90CF90BF9008950E94751188E1E3EAB4
:10241000F2E0DF01982F1D929A95E9F7EBE8F2E0E0
:10242000DF011D928A95E9F78CE00E9464120C94FA
:102430000203FF920F931F93CF93DF93CDB7DEB7C5
:1024400068970FB6F894DEBF0FBECDBF8E010F5F49
:102450001F4F88E1F80111928A95E9F7F12C6F2D51
:10246000C8010E949511F394FCE0FF12F8CF48E1F7
:1024700050E0B8018BE892E00E943C20FF24F394E6
:10248000009709F4F12C892B41F088E1F801ABE8C1
:10249000B2E001900D928A95E1F72F2D4CE063EAAE
:1024A00072E08BE892E00E9465120E9404038F2D77
:1024B00068960FB6F894DEBF0FBECDBFDF91CF9107
:1024C0001F910F91FF9008950895FF920F931F930E
:1024D000CF93DF93F82E092F162FD72FC42F222347
:1024E00049F081E0809362020E94C31890936102D8
:1024F00080936002809162028823D9F0809160020B
:10250000909161020E94DB18059798F0EF2DF02F53
:10251000A12FBD2F80E090E04C2F50E0841795074D
:1025200034F4219131912D933D930196F7CF109280
:102530006202DF91CF911F910F91FF9008950E9449
:10254000D41A0E94580E0C94E01A0E94E41A0E94B9
:10255000FB0E0C94FE1A0E9461180E94BB1A0E9486
:10256000460E0E949F120E94A5120E94500EFBCFA1
:102570008091690280FF06C06091090170E0660FDA
:10258000771F26C081FF04C06091090184E005C067
:1025900082FF07C06091090188E0689FB0011124A3
:1025A00017C0909168029923D1F0609108019617A5
:1025B00088F72091090188E0289F90011124929FBB
:1025C000A001939F500D112470E0CA010E940E20BB
:1025D0006038710540F46115710519F406C068E0B2
:1025E00070E0862F08958FE7089581E00895809127
:1025F000690280FF08C06091050170E075956795DC
:102600007595679521C081FF06C06091050170E056
:102610007595679519C082FF04C06091050170E04F
:1026200010C090916702992399F060910401961768
:10263000A0F780910501899FC001112470E00E94DC
:102640000E206038710540F46115710519F406C05B
:1026500061E070E0862F08958FE7089581E0089586
:102660008D3E21F40E94B812819504C08E3E29F45B
:102670000E94B81280936D0208958F3E21F40E944B
:10268000B812819504C0803F29F40E94B81280934B
:102690006C020895893F19F40E94F71205C08A3F21
:1026A00031F40E94F712819580936E0208958B3F5A
:1026B00021F40E94F712819504C08C3F29F40E94F6
:1026C000F71280936F0208959FE0980F983078F486
:1026D00021E030E0A90102C0440F551F9A95E2F7AE
:1026E000CA0190916B02892B80936B0208958D3FF4
:1026F00021F48091690281600BC08E3F21F48091AA
:102700006902826005C08F3F29F48091690284606C
:102710008093690208958D3E39F490916D0297FF80
:1027200035C010926D0259C08E3E29F490916D0211
:102730001916BCF32BC090916C028F3E29F497FFC1
:1027400025C010926C0249C0803F19F41916CCF3D1
:102750001DC090916E02893F29F41916BCF41092A5
:102760006E023BC08A3F19F497FF10C0F8CF8B3F31
:1027700039F490916F0297FF09C010926F022DC03B
:102780008C3F21F490916F021916BCF39FE0980FD3
:10279000983080F421E030E0A90102C0440F551FB9
:1027A0009A95E2F7CA01809590916B0289238093F4
:1027B0006B0213C08D3F21F4809169028E7F0BC0A4
:1027C0008E3F21F4809169028D7F05C08F3F29F4EF
:1027D000809169028B7F8093690280916C028111E4
:1027E00006C080916D02811102C010926802809132
:1027F0006E02811106C080916F02811102C0109299
:10280000670208950E94C31820916C02211104C030
:1028100020916D02222321F090936602809365023D
:1028200020916E02211104C020916F02222321F019
:1028300090936402809363028AE692E00C94A0175E
:10284000EF92FF920F931F93CF93DF9300D000D0AE
:1028500000D0CDB7DEB786E0EAE6F2E0DE01119601
:1028600001900D928A95E1F7E0906C02F0906D0274
:1028700000916E0210916F0210926C0210926D0224
:1028800010926E0210926F02E11003C0FF2009F453
:102890005DC080916502909166020E94DB18AC01D8
:1028A00090916802992339F020910A0130E02417B1
:1028B000350758F04BC020910B018AE0289F90010A
:1028C00011242417350718F041C09F3F19F09F5F6E
:1028D00090936802EE2061F00E94B8121E1414F06A
:1028E0009FEF01C091E0989F902D112490936C026E
:1028F000FF2061F00E94B8121F1414F09FEF01C076
:1029000091E0989F902D112490936D0230916C026C
:102910003323E1F020916D022223C1F045EB340313
:10292000C0011124992319F090936C0203C081E037
:1029300080936C0235EB2303C0011124992319F015
:1029400090936D0203C081E080936D02011103C07A
:10295000112309F45DC080916302909164020E948A
:10296000DB18AC0190916702992339F020910601A0
:1029700030E02417350758F04BC0209107018AE05A
:10298000289F900111242417350718F041C09F3F5C
:1029900019F09F5F90936702002361F00E94F71285
:1029A000101614F09FEF01C091E0989F902D112414
:1029B00090936E02112361F00E94F712111614F029
:1029C0009FEF01C091E0989F902D112490936F028A
:1029D00030916E023323E1F020916F022223C1F087
:1029E00045EB3403C0011124992319F090936E0232
:1029F00003C081E080936E0235EB2303C0011124F4
:102A0000992319F090936F0203C081E080936F02C5
:102A100080916C0281110BC080916D02811107C001
:102A200080916E02811103C080916F0281110E941A
:102A30000214EB82FC820D831E8386E0FE01319638
:102A4000AAE6B2E001900D928A95E1F726960FB6BC
:102A5000F894DEBF0FBECDBFDF91CF911F910F91D4
:102A6000FF90EF900895EAE6F2E086E0DF011D9224
:102A70008A95E9F710926802109267021092690233
:102A80000895CF93DF93EC01FB018281882309F441
:102A90003CC1C430FDE5DF0760F4CB3F9CE5D907BE
:102AA00088F49E0122503C452431310508F02EC1A6
:102AB00009C0C236EDE5DE0729F0C63AFDE5DF07BD
:102AC00009F024C10E947F0D90938A0280938902AD
:102AD000C1318CE5D80709F4C6C008F042C0C9303E
:102AE000ECE5DE0709F49BC000F5C5308CE5D8079E
:102AF00009F485C078F4C330ECE5DE0709F478C04A
:102B000008F07AC0C230DC4509F0F5C08091890236
:102B10008160EFC0C7309CE5D90709F478C008F0A0
:102B20007AC0809189028061E4C0CD30FCE5DF0786
:102B300009F487C058F4CB309CE5D90709F479C073
:102B400008F07BC08091890288606FC0CF30FCE5BF
:102B5000DF0709F480C008F082C080918902877F76
:102B6000C8C0CE3F9CE5D90709F471C000F5C53156
:102B7000FCE5DF0709F485C068F4C3319CE5D9079B
:102B800009F475C008F095C00E9430078091890251
:102B90008F77AFC0CC3FFCE5DF07A9F108F054C048
:102BA000CB3FDC4509F0A7C080918A0240C0C2300B
:102BB000EDE5DE0709F489C058F4C1158DE5D807A5
:102BC00009F45AC008F069C080918A0282602FC05F
:102BD000C236EDE5DE0709F47CC0C63AFDE5DF0745
:102BE00009F481C0C330DD4509F085C080E06EC0C6
:102BF0008091890282607DC08091890216C0809197
:102C00008902886076C080918A0282604FC080917C
:102C1000890280626EC08091890280646AC00E94CD
:102C2000300780918902806864C0846062C08160DE
:102C30003DC0809189028E7F5CC0809189028D7F2A
:102C400058C08091890216C080918A0218C0809174
:102C50008A028D7F2BC0809189028F7E4AC080912D
:102C600089028F7D46C0809189028F7B42C080910E
:102C70008902877F8B7F3DC080918A028D7F8E7F06
:102C800015C08091890282FB222720F991E09227CA
:102C900090FB82F990FB83F92CC080918A02982FD7
:102CA000909591708E7F892B90FB81F980938A0299
:102CB00022C00E9430078091890287FB222720F9D9
:102CC00091E0922790FB87F914C081E00E94160ED4
:102CD00012C08091890284FB222720F991E092277B
:102CE00090FB84F906C080918902982F909590FB03
:102CF00080F9809389028091890290918A020E94D2
:102D0000900D0E94300780E001C081E0DF91CF91FB
:102D10000895CF93DF9386319C4541F5EB010E94E6
:102D2000830C982F8A81209102013091030188231E
:102D300079F09A7A81E009F480E080937002911131
:102D400002C069E201C065E3C9010E941C180AC003
:102D500080917002811102C069E201C065E3C9017E
:102D60000E941E180E94C50C80E001C081E0DF9126
:102D7000CF9108950F931F93CF93DF93C42FD22F3A
:102D8000FC0182818823C9F0409373020E94C3181A
:102D9000909372028093710280E28C0F883008F069
:102DA00057C0C77081E001C0880FCA95EAF7DF916C
:102DB000CF911F910F910C948D0480917302481351
:102DC00030C080917102909172020E94DB18883CA1
:102DD000910538F510E21D0FCD17B9F080E28C0F88
:102DE000883040F4C77081E001C0880FCA95EAF7C7
:102DF0000E949404183028F581E09D2F977001C03F
:102E0000880F9A95EAF70E948D04802F0E9484040F
:102E10001830F0F4D77081E001C0880FDA95EAF736
:102E20000AC080E28C0F883098F4C77081E001C03E
:102E3000880FCA95EAF7DF91CF911F910F910C94FB
:102E40009404802FDF91CF911F910F910C948404F3
:102E5000DF91CF911F910F9108950F939C01CB01AA
:102E6000243F4CE5340731F188F4293DFCE53F0768
:102E7000D9F02A3D4CE5340779F1283D3C45A9F5C8
:102E800006E221EE41EE68ED7CE52BC0263FFCE535
:102E90003F07E1F0A8F0273F3C4539F507E225EE72
:102EA00046EE67EF7CE51DC007E225EE45EE69EDD5
:102EB0007CE517C006E221EE40EE64EF7CE511C030
:102EC00007E225EE44EE65EF7CE50BC006E221EE5D
:102ED00042EE66EF7CE505C008E221E045EE6AEDD2
:102EE0007CE50E94BA1680E008C0FC01828188233C
:102EF00019F01092730201C081E00F910895909330
:102F000093018093920108959093790280937802BF
:102F10000895E0917802F0917902309721F00190C4
:102F2000F081E02D099480E00895E0917802F0911D
:102F30007902309721F00280F381E02D0994089501
:102F4000E0917802F0917902309739F022E0DC01CB
:102F50002C930480F581E02D099408952091760248
:102F6000309177022817390771F090937702809398
:102F70007602E0917802F0917902309721F0068094
:102F8000F781E02D09940895209174023091750223
:102F90002817390771F09093750280937402E091BD
:102FA0007802F0917902309721F00084F185E02DCC
:102FB00009940895FC01329697E080E0915029F041
:102FC00021912223D9F38F5FF9CF0895662349F029
:102FD000FC01329608962191621729F0E817F9074B
:102FE000D1F780E0089581E008959C01FC013296BC
:102FF0009FEF80E04191461789F09F3F19F44111FE
:1030000001C0982F8F5F8630A9F79F3F39F0F901F3
:10301000E90FF11D97FDFA956283089508959C01CB
:103020002A5F3F4FFC014281461301C01282019684
:1030300082179307B9F708950C94F5170C940F189D
:10304000029626E0FC0111922A95E9F70895089569
:103050000C94271883E080937A020C94281881112D
:1030600002C081E001C082E080937A020C942818AB
:103070000C942F1881E080937A020C9428180C94F9
:103080003A1808950C9441180C9442180C94411865
:103090000C9441180C944118CF930E9448180E9438
:1030A00019120E944618C0E08C2F0E944311892BF0
:1030B00029F4CF5FCC30C1F780E001C081E0CF912F
:1030C000089508951F920F920FB60F9211248F93B7
:1030D0009F93AF93BF9380917B02811113C0809126
:1030E000BB029091BC02A091BD02B091BE0241967C
:1030F000A11DB11D8093BB029093BC02A093BD02A1
:10310000B093BE02BF91AF919F918F910F900FBE70
:103110000F901F9018958091C302843031F10E9466
:10312000680310927B0220E488E190E00FB6F894E7
:10313000A895809360000FBE2093600083B7817FC5
:10314000846083BF83B7816083BF7894889583B799
:103150008E7F83BF0FB6F894A89580916000886138
:1031600080936000109260000FBE08950E943007A7
:103170000C946C0382E084BD93E095BD9AEF97BDFB
:1031800080936E0008952FB7F8948091BB029091C0
:10319000BC02A091BD02B091BE022FBF08952FB70F
:1031A000F8946091BB027091BC028091BD02909135
:1031B000BE022FBF08959C014FB7F8948091BB02C7
:1031C0009091BC02A091BD02B091BE024FBF821B84
:1031D000930B089578941F920F920FB60F921124BB
:1031E0008F939F93AF93BF938091BB029091BC024A
:1031F000A091BD02B091BE020196A11DB11D8093A8
:10320000BB029093BC02A093BD02B093BE02BF91DB
:10321000AF919F918F910F900FBE0F901F901895B7
:10322000F89481E08093E00080E28093D800E9EC9C
:10323000F0E010828FE19EE40197F1F700C00000FA
:103240001DBA109268001CBC10BE1FBA10927A0002
:1032500010926E0010926F00109271001092720026
:103260001082ECEBF0E0108214B817B81AB81DB851
:1032700010BA108215B818B81BB81EB811BA0C9441
:10328000003F0895809187020895089522E02093D9
:10329000E9002FEF3091E800215035FD06C035EDF3
:1032A0003A95F1F700002111F5CF2091E80025FFB4
:1032B0000BC040E050E066E070E00E94701B80911F
:1032C000E8008E778093E8000895CF93DF9321E0A4
:1032D0002093E9002FEF3091E800215035FD06C022
:1032E00035ED3A95F1F700002111F5CF2091E80076
:1032F00025FF14C0EC0140E050E068E070E00E945F
:10330000701B8091E8008E778093E80088E0FE01D2
:10331000AFE7B2E001900D928A95E1F7DF91CF918E
:10332000089580937C0270937E0260937D02809169
:10333000C302843001F582E08093E9008FEF909121
:10334000E800815095FD06C095ED9A95F1F70000D3
:103350008111F5CF8091E80085FF0DC040E050E07D
:1033600063E070E08CE792E00E94701B8091E800BF
:103370008E778093E8000895BC0184E00C94911945
:10338000BC0183E00C9491198091C202811109C0A3
:103390000E94011D0E945E1D8091E2008460809366
:1033A000E20008951092C20208950C943F186091B3
:1033B000BF0281E0611101C080E00C942A18909155
:1033C000C30281E0943009F080E06091BF020C9468
:1033D0002F1842E061EC81E00E947A1C42E261EC2D
:1033E00082E00E947A1C9091C30281E0943009F03F
:1033F00080E06091BF020C9438188091C502833040
:1034000009F461C030F4813071F0823009F49AC05F
:1034100008958A3009F486C08B3009F46CC0893075
:1034200009F0A8C020C08091C402813A09F0A2C06E
:103430008091E800877F8093E8008091C802909196
:10344000C902892B21F468E08FE792E003C060E0B5
:1034500080E090E070E00E94BB1B8091E8008B77D9
:103460008093E80008958091C402813209F082C0FF
:103470008091C8029091C902029708F07BC08091A8
:10348000E800877F8093E8008091E80082FD05C016
:103490008091C3028111F8CF6DC02091F30080911B
:1034A000F20090E0922B029731F48091F10081308C
:1034B00011F0863021F48091F10080938702809191
:1034C000E8008B7753C08091C402813A09F052C062
:1034D0008091C8029091C902892B09F04BC080915C
:1034E000E800877F8093E8008091E80080FFFCCFB0
:1034F0008091180136C08091C4028132D9F5809143
:10350000C8029091C902892BA9F58091E800877FB4
:103510008093E8000E94AF1C8091C602809318013E
:103520000C9430078091C402813221F58091E8002B
:10353000877F8093E8000E94AF1C8091C702809330
:10354000880208958091C402813AA1F48091E80034
:10355000877F8093E8008091E80080FFFCCF809116
:1035600088028093F1008091E8008E778093E800D4
:103570000C94AF1C089584B7877F84BF0FB6F8946E
:10358000A89580916000886180936000109260002F
:103590000FBE90E080E80FB6F8948093610090939E
:1035A00061000FBE0C943A180E94011D0E945E1D1E
:1035B000E2EEF0E080818460808378940C94F31FC5
:1035C0008CE091E00C9484178091C3028530A9F4BB
:1035D0008091C302853079F40E948B188091C102DA
:1035E0008823B1F30E944C18882391F30E945A1B40
:1035F0000E943007EDCF0C94B618089508950C94EE
:10360000011B292F332723303105C9F060F4213005
:10361000310581F02230310509F044C08BE390E0A0
:103620002AE134E043C021323105E1F02232310594
:1036300049F138C082E190E025E534E037C09927B0
:103640008130910549F028F0029761F5E0EFF3E051
:1036500005C0E6E1F4E002C0EEE0F4E0849190E021
:103660009F0124C06115710541F061307105D1F4ED
:1036700089E090E025E434E019C089E090E02CE294
:1036800034E014C06115710541F06130710551F4E9
:103690008BE790E027E634E009C080E490E022EE7A
:1036A00034E004C080E090E020E030E0FA013183B3
:1036B0002083089580E189BD82E189BD09B400FEBF
:1036C000FDCF8091D8008F7D8093D8008091E0005D
:1036D00082608093E0008091E00081FDFCCF08953E
:1036E000CF92DF92EF92FF920F931F93CF93DF93CE
:1036F000EC018B017A010E94CE1C811133C0E114D0
:10370000F10439F0F70180819181081B190BC80F72
:10371000D91FC12CD12C0115110519F18091E80098
:1037200085FD16C08091E8008E778093E800E11453
:10373000F10449F0F70180819181C80ED91ED18230
:10374000C08285E00FC00E94CE1C882321F30AC0EE
:1037500089918093F10001501109FFEFCF1ADF0A20
:10376000DACF80E0DF91CF911F910F91FF90EF9022
:10377000DF90CF9008952091CA023091CB02261796
:10378000370748F06115710539F42091E8002E776C
:103790002093E80001C0B901FC0120E0611571052A
:1037A00079F18091C3028823F1F18530F1F18091A4
:1037B000E80083FD3CC08091E80082FD2EC080912E
:1037C000E80080FFEBCF2091F3008091F20090E0C1
:1037D000922B6115710551F08830910538F42191D3
:1037E0002093F100615071090196F3CF21E0089711
:1037F00009F020E08091E8008E778093E800CECF3A
:103800002111CFCF0AC08091C302882361F0853097
:1038100061F08091E80083FD0AC08091E80082FF9A
:10382000F2CF80E0089582E0089583E0089581E07A
:1038300008952091CA023091CB022617370748F02D
:103840006115710539F42091E8002E772093E80086
:1038500001C0B901FC0120E06115710591F1809171
:10386000C302882309F440C0853009F43FC0809129
:10387000E80083FD3DC08091E80082FD2FC080916B
:10388000E80080FFE9CF2091F3008091F20090E002
:10389000922B6115710559F08830910540F42491FF
:1038A0002093F1003196615071090196F2CF21E029
:1038B000089709F020E08091E8008E778093E80077
:1038C000CBCF2111CCCF0AC08091C302882361F0F5
:1038D000853061F08091E80083FD0AC08091E800A6
:1038E00082FFF2CF80E0089582E0089583E008959A
:1038F00081E00895982F973068F59093E900981724
:1039000039F07091EC002091ED005091F00003C06F
:10391000242F762F50E021FD02C09F5FECCF309125
:10392000EB003E7F3093EB003091ED003D7F309314
:10393000ED003091EB0031603093EB007093EC00C0
:103940002093ED005093F0002091EE0027FDE5CF8D
:1039500080E008958F708093E90081E00895809160
:10396000C40287FF11C08091E80082FD05C08091EC
:10397000C3028111F8CF11C08091E8008B770BC092
:103980008091C302882349F08091E80080FFF8CF3E
:103990008091E8008E778093E80008952091E400FC
:1039A0003091E50095E64091EC00842F817040FF56
:1039B00023C08091E80080FD1DC08091C302882350
:1039C00099F0853099F08091EB0085FD11C0409110
:1039D000E4005091E5002417350729F3915011F0C8
:1039E0009A01E1CF84E0089582E0089583E008958C
:1039F00081E0089580E008954091E80042FFDDCF26
:103A000008950E946F1D0E94771DE0EEF0E0808116
:103A100081608083E8EDF0E080818F77808319BC3E
:103A2000A7EDB0E08C918E7F8C9380818F7E808318
:103A30001092C20208950F931F93CF93DF930E94B9
:103A40006F1D0E94771DC8EDD0E088818F77888335
:103A500088818068888388818F7D888319BC1092D3
:103A6000C3021092BF021092C1021092C00200EE77
:103A700010E0F80180818B7F80838881816088835A
:103A800042E060E080E00E947A1CE1EEF0E080819C
:103A90008E7F8083E2EEF0E0808181608083808190
:103AA00088608083F80180818E7F80838881806137
:103AB0008883DF91CF911F910F910895E8EDF0E099
:103AC00080818F7E8083E7EDF0E08081816080835C
:103AD00084E082BF81E08093C2020C941B1DE8ED5C
:103AE000F0E080818E7F80831092E2000895109232
:103AF000DA001092E10008951F920F920FB60F9214
:103B000011242F933F934F935F936F937F938F93E2
:103B10009F93AF93BF93EF93FF938091E10082FF58
:103B20000BC08091E20082FF07C08091E1008B7F93
:103B30008093E1000E94F21F8091DA0080FF1FC095
:103B40008091D80080FF1BC08091DA008E7F809327
:103B5000DA008091D90080FF0DC080E189BD82E14B
:103B600089BD09B400FEFDCF81E08093C3020E94AD
:103B7000C41905C019BC1092C3020E94D2198091C9
:103B8000E10080FF19C08091E20080FF15C08091A4
:103B9000E2008E7F8093E2008091E200806180935A
:103BA000E2008091D80080628093D80019BC85E043
:103BB0008093C3020E94D7198091E10084FF30C036
:103BC0008091E20084FF2CC080E189BD82E189BD43
:103BD00009B400FEFDCF8091D8008F7D8093D8007E
:103BE0008091E1008F7E8093E1008091E2008F7EE2
:103BF0008093E2008091E20081608093E2008091F6
:103C0000BF02882311F084E007C08091E30087FDA4
:103C100002C081E001C083E08093C3020E94DF19EB
:103C20008091E10083FF29C08091E20083FF25C0DD
:103C30008091E100877F8093E10082E08093C3025E
:103C40001092BF028091E1008E7F8093E10080910D
:103C5000E2008E7F8093E2008091E2008061809399
:103C6000E20042E060E080E00E947A1C8091F00077
:103C700088608093F0000E94D519FF91EF91BF9169
:103C8000AF919F918F917F916F915F914F913F91F4
:103C90002F910F900FBE0F901F9018951F920F92AB
:103CA0000FB60F9211242F933F934F935F936F930F
:103CB0007F938F939F93AF93BF93CF93DF93EF93B4
:103CC000FF93C091E900CF708091EC00D82FD170A4
:103CD00080FDD0E81092E9008091F000877F80930A
:103CE000F00078940E94921E1092E9008091F000FA
:103CF00088608093F000CD2BCF70C093E900FF91D6
:103D0000EF91DF91CF91BF91AF919F918F917F9173
:103D10006F915F914F913F912F910F900FBE0F9038
:103D20001F9018951F93CF93DF93CDB7DEB7AA9757
:103D30000FB6F894DEBF0FBECDBFE4ECF2E0809189
:103D4000F100819322E0EC3CF207C9F70E94FD19D3
:103D50008091E80083FF2EC18091C4029091C5023A
:103D6000492F50E04A30510508F024C1FA01EE59BC
:103D7000FF4F0C942220803821F0823809F01AC1BC
:103D800008C08091C0029091C102992389F082609D
:103D90000FC08091C8028F70873008F00BC18093EC
:103DA000E9008091EB0085FB882780F91092E900FB
:103DB0009091E800977F9093E8008093F100109233
:103DC000F100D1C0282F2D7F09F0F4C0882319F00D
:103DD000823061F0EFC08091C602813009F0EAC004
:103DE000933009F080E08093C1022EC08091C6021A
:103DF00081112AC08091C8028F702FEF280F2630C2
:103E000008F0D8C08093E9002091EB0020FF1CC08F
:103E1000933021F48091EB00806214C09091EB000C
:103E200090619093EB0021E030E0A90102C0440FC3
:103E3000551F8A95E2F74093EA001092EA008091BC
:103E4000EB0088608093EB001092E9008091E8001D
:103E5000877F8093E8000E94AF1CACC08111AAC08C
:103E60001091C6021F778091E3008078812B8093A8
:103E7000E3008091E800877F8093E8000E94AF1CF8
:103E80008091E80080FFFCCF8091E3008068809300
:103E9000E300111102C082E001C083E08093C302FD
:103EA00089C08058823008F085C08091C602909108
:103EB000C7028C3D53E0950779F583E08A838AE257
:103EC00089834FB7F894DE01139620E03EE051E27B
:103ED000E32FF0E050935700E49120FF03C0E295F8
:103EE000EF703F5FEF708E2F90E0EA3010F0C796D2
:103EF00001C0C0968D939D932F5F243149F74FBF2A
:103F00008091E800877F8093E8006AE270E0CE014C
:103F100001960E94BB1B16C06091C8027091C90235
:103F2000AE014F5F5F4F0E94FF1ABC01892B09F45D
:103F300041C09091E800977F9093E80089819A8131
:103F40000E94191C8091E8008B778093E80032C0B2
:103F5000803881F58091E800877F8093E800809128
:103F6000BF028093F1008091E8008E7772CF8111BB
:103F700021C08091C6029091C70299270297D4F47C
:103F80008091E800877F8093E8008091C60280934B
:103F9000BF020E94AF1C8091BF02811106C08091B8
:103FA000E30087FD02C081E001C084E08093C3028A
:103FB0000E94E9198091E80083FF0AC08091E8001F
:103FC000877F8093E8008091EB0080628093EB0014
:103FD000AA960FB6F894DEBF0FBECDBFDF91CF918A
:103FE0001F9108950895CF938091C3028823A1F073
:103FF000C091E900CF709091EC00892F817090FD05
:1040000080E8C82B1092E9008091E80083FD0E94AF
:10401000921ECF70C093E900CF91089597FB072EB1
:1040200016F4009407D077FD09D00E94282007FCE1
:1040300005D03EF4909581959F4F089570956195B8
:104040007F4F0895EE0FFF1F0590F491E02D099426
:10405000AA1BBB1B51E107C0AA1FBB1FA617B707AE
:1040600010F0A61BB70B881F991F5A95A9F78095CA
:104070009095BC01CD010895FB01DC0104C08D9138
:104080000190801921F441505040C8F7881B990BCA
:104090000895F999FECF92BD81BDF89A992780B510
:1040A0000895A8E1B0E042E050E00C947D20262F76
:1040B000F999FECF92BD81BDF89A019700B402161E
:1040C00039F01FBA20BD0FB6F894FA9AF99A0FBECC
:1040D00008950396272F0E9458200E945720252FCD
:1040E0000E945820242F0C9458200196272F0E94BC
:1040F00058200C945720DC01CB01FC01F999FECF2C
:1041000006C0F2BDE1BDF89A319600B40D9241505F
:0A4110005040B8F70895F894FFCF6F
:10411A00C8003502280850011E0A140142196519FF
:10412A004619C019BC19451901E200E900EA00B5AF
:10413A0000B600B700CD008301CC008A0192019439
:10414A00012102230224022502260227022A02B39F
:10415A0000B4006F007000818283E200E900EA0087
:10416A00B500B600B700CD008301CC008A019201E8
:10417A0094012102230224022502260227022A028E
:10418A00B300B4006F0070008182839192936695A8
:10419A00679497343536303132333790F0F1F4F58D
:0241AA00F6F726
:00000001FF
